:020000023000CC
:10E000000D949AF00D94C3F00D94C3F00D94C3F0E9
:10E010000D94C3F00D94C3F00D94C3F00D94C3F0B0
:10E020000D94C3F00D94C3F00D94C3F00D94C3F0A0
:10E030000D94C3F00D94C3F00D94C3F00D94C3F090
:10E040000D94C3F00D94C3F00D94C3F00D94C3F080
:10E050000D94C3F00D94C3F00D94C3F00D94C3F070
:10E060000D94C3F00D94C3F00D94C3F00D94C3F060
:10E070000D94C3F00D94C3F00D94C3F00D94C3F050
:10E080000D94C3F00D94C3F00D94C3F00D94C3F040
:10E090000D94C3F00D94C3F00D94C3F00D94C3F030
:10E0A0000D94C3F00D94C3F00D94C3F00D94C3F020
:10E0B0000D94C3F00D94C3F00D94C3F00D94C3F010
:10E0C0000D94C3F00D94C3F00D94C3F00D94C3F000
:10E0D0000D94C3F00D94C3F00D94C3F00D94C3F0F0
:10E0E0000D94C3F00D94C3F00D94C3F00D94C3F0E0
:10E0F0000D94C3F00D94C3F00D94C3F00D94C3F0D0
:10E100000D94C3F00D94C3F00D94C3F00D94C3F0BF
:10E110000D94C3F00D94C3F00D94C3F00D94C3F0AF
:10E120000D94C3F00D94C3F00D94C3F00D94C3F09F
:10E130000D94C3F011241FBECFEFD1E8DEBFCDBFD9
:10E1400001E00CBF12E0A0E0B2E0E6E3F8EE03E08D
:10E150000BBF02C007900D92A430B107D9F722E09F
:10E16000A4E0B2E001C01D92A630B207E1F70F941F
:10E17000E0F00D9419F401E80EBF0FEF0DBF11246C
:10E180001FBE0D94E0F00D9400F08093C6008091C6
:10E19000C00086FFFCCF8091C00080648093C000E7
:10E1A000089520E030E02817390749F0EFECF7E058
:10E1B0003197F1F700C000002F5F3F4FF4CF089573
:10E1C000CF93DF93CDB7DEB7C352D1400FB6F894EB
:10E1D000DEBF0FBECDBF80E880936100109261006A
:10E1E00001E80EBF0FEF0DBF84B78EBBF894A89562
:10E1F00014BE80916000886180936000109260007E
:10E2000078946B9A739A22981092C0001092C10071
:10E210008091C6008091C00082608093C00093E32B
:10E220009093C40088E18093C1008091C000826017
:10E230008093C0009093C40000008CB1C12CD12CFD
:10E24000760167EC862E6BE1962EA12CB12C78E03E
:10E25000772E00E010E08091C00087FF04C00F5FC0
:10E260001F4FB9F326C001151105C9F725E02A95FE
:10E27000F1F700008FEFC81AD80AE80AF80A91E00F
:10E2800080E0A1E6CA16AAEEDA06E104F10408F479
:10E2900090E0092F182FC701B601A50194010F9432
:10E2A000E9F3672B682B692BB1F68EB187258EB900
:10E2B000D2CF0130110509F070C2C25EDE4F188264
:10E2C000CE51D140512C212C312C812C912C540138
:10E2D000C12CD12C760120E030E060E00130110546
:10E2E000B9F081E092E1AAE7B0E04091C00047FDBB
:10E2F0000FC00197A109B109C1F7ABBFFC0147915C
:10E3000056914F3F5F4F69F3EE27FF270994E9CFFE
:10E310004091C600633001F120F4613071F038F0B3
:10E3200014C0653029F1E0F0663099F135C04B3109
:10E3300009F447C200E010E0D1CF5426C25EDE4FA0
:10E340004883CE51D14062E0F5CF242F30E0322F08
:10E350002227542663E0EECF242B542664E0EACF34
:10E360004E3009F032C25426212C312C65E0E2CF28
:10E37000C1010196E1E0F0E0EC0FFD1FE20DF31D9D
:10E38000408354268217930709F021C2190166E0E1
:10E39000D1CF45111AC202C0673061F649814331BD
:10E3A00009F4DDC068F5463009F4C7C000F5423015
:10E3B00009F479C0433009F466C0413009F09BC1CB
:10E3C0001A8288E08B8381E48C8386E58D8382E5E5
:10E3D0008E8389E48F8383E5888780E589878FE54D
:10E3E0008A8782E38B87412C0BE010E089C14131A1
:10E3F00009F456C008F099C0403109F454C07BC1FB
:10E40000483109F46BC048F4453109F4A8C008F458
:10E4100028C1463109F425C16EC14A3109F451C001
:10E4200008F471C04B3109F441C04D3109F063C1AA
:10E430009D81903339F48F818823B1F08130B1F020
:10E4400082E017C0892F807599F0903521F489E01A
:10E45000E0E0F0E005C0983559F4E3E0F0E089E051
:10E4600080935700849105C08EE103C088EA01C003
:10E4700080E01A821B829C831D828E831F82412C26
:10E4800007E010E03DC1EA81E059E33028F4F0E014
:10E49000E050FE4F808101C080E01A828B8341C032
:10E4A0004424439401C0412C1A8228C18D818823C1
:10E4B00021F0813021F082E024C08EE122C088EA80
:10E4C00020C01A82E1E0F0E089E080935700849157
:10E4D0008B831C82412C04E010E012C18B818035BB
:10E4E00051F48C81883019F4E2E0F0E006C089E054
:10E4F000E0E0F0E003C0E3E0F0E089E08093570063
:10E5000084911A82E5CF8D81836C99E0E1E0F0E09F
:10E51000082E90935700E89507B600FCFDCF1A82AD
:10E520001B82412C03E010E0EBC01A82412C02E078
:10E5300010E0812C912C5401E3C08A81CB80D12C36
:10E54000E12CF12C7601DD24CC24F82A8D81C82A17
:10E550008C81D82ACC0CDD1CEE1CFF1C80C02A81CB
:10E5600030E0322F22278B812901482A433109F0DC
:10E5700044C08114F0EC9F06F3E0AF06B10470F4E0
:10E5800083E0F401A0925B0080935700E89507B602
:10E5900000FCFDCF2FEF921AA20AB20A8B85B701B9
:10E5A000A601DE011B9611E01296FD013197E08174
:10E5B00090E09E2B0C01FA0160935B0010935700D2
:10E5C000E89511244E5F5F4F6F4F7F4F82E0481AEE
:10E5D000510811F08C91E8CF85E0F601E0925B00E4
:10E5E00080935700E89507B600FCFDCF81E180934A
:10E5F0005700E8956A017B0132C0D701C601B69584
:10E60000A79597958795C15EDE4F88839983AA83E6
:10E61000BB83CF51D1408E01055F1F4F612C712C00
:10E620006414750489F0D8016D918D01C15EDE4FCF
:10E6300088819981CF51D140860D971D0F940BF49D
:10E64000BFEF6B1A7B0AECCFC301A0E0B0E0880FEC
:10E65000991FAA1FBB1FC80ED91EEA1EFB1E1A82D5
:10E660004CC08A8190E0982F88272B81822B8C01C7
:10E670000D5F1F4F1A82443199F4DE011396EBBEF1
:10E68000F601279136912C931296FD013197308334
:10E69000E2E0CE0ED11CE11CF11C029781F728C0EC
:10E6A000FE0133969C01B701A60141BD452E562EB1
:10E6B000672E772442BC4F5F5F4F6F4F7F4FF89AB2
:10E6C000A0B5A1932150310981F7AC014150510906
:10E6D00060E070E04F5F5F4F6F4F7F4FC40ED51EFD
:10E6E000E61EF71EA3E0B0E0AC0FBD1FA80FB91FD8
:10E6F0001C92412C05C080EC8A83412C02E010E082
:10E700008BE10F94C5F0C25EDE4F8881CE51D140BF
:10E710000F94C5F0812F0F94C5F0802F0F94C5F092
:10E7200085E1C25EDE4F5880CE51D140582650263A
:10E730008EE00F94C5F05126CE0101963C01080FE2
:10E74000191F6016710691F0F30191913F01892F15
:10E75000CD5DDE4F9883C352D1400F94C5F0CD5D9F
:10E76000DE4F9881C352D1405926EBCF852D0F94AF
:10E77000C5F0C25EDE4F2881CE51D1402F5FC25E10
:10E78000DE4F2883CE51D1409EB188E089278EB9D3
:10E7900000E010E0442009F49ECD6B98739884E665
:10E7A00090E00F94D1F000008091C0008D7F8093A5
:10E7B000C00081E180935700E895EE27FF27099478
:10E7C000FFCF8BE1582E61E0B5CD60E0B3CD1C01E9
:10E7D000B1CDA1E21A2EAA1BBB1BFD010DC0AA1FC1
:10E7E000BB1FEE1FFF1FA217B307E407F50720F0BA
:10E7F000A21BB30BE40BF50B661F771F881F991F35
:10E800001A9469F760957095809590959B01AC017D
:10E81000BD01CF010895262FF999FECF1FBA92BDF1
:10E8200081BD20BD0FB6F894FA9AF99A0FBE0196F1
:06E830000895F894FFCFEB
:04E836000F020A00C3
:040000033000E000E9
:00000001FF
